:020000040000FA
:060000002FEF27F01200B3
:0600080012EF20F01200CF
:06002A000200964E0000EA
:1000300014010000080000007C4E000000000000D9
:040040001A000000A2
:0C0044000E0EC16E010EC26E860EC06E64
:1000500084B603D00101010E156F0001EA6BEB6B52
:100060008A6A896AF90E926EBA6ABD6A010E066ED4
:10007000640EEC6FD00EEF6F070EF06F080EED6F91
:100080000B0EEE6F000E036E046A096E0A6A076EAD
:10009000086A800ED56E1200F2A418D0F294000106
:1000A000EB2B050E0101005D07E20A0E0001EB5D7E
:1000B00003E38974EB6B1200050E0101005D06E19C
:1000C0002E0E0001EB5D02E38974EB6B1200E4DF9E
:1000D000050E0101005D66E36D50020B01E01200A8
:1000E0000001EA5129E0800E04010C1525E1400EC3
:1000F000E66E600EE66E000EE66E48EC21F0E5520C
:10010000E552E5520001EA6B016A0250015C13E21C
:100110000150EA6AE00FE96E000EEA22EF50E66E47
:100120000150EA6A600FE96E000EEA22E552E750DC
:10013000EF6E012AEAD7026A01011451005C31E333
:1001400001501FE0400E015C09E20150EA6A600FB5
:10015000E96E000EEA22EF6A012AF4D7016A04016F
:100160000CBF0CD0400EE66E600EE66E000EE66E22
:1001700048EC21F0E552E552E55203D00001010EB2
:10018000EA6F400EE66EA00EE66E000EE66E8AEC9A
:1001900021F0E552E552E5520101146FE85001E00B
:1001A000006A01D81200D9CFE6FFE1CFD9FF100EC7
:1001B000E12601011451005C02E3D2EF1FF00001BF
:1001C000EA5102E0D2EF1FF089820050EA6AA00FE4
:1001D000E96E000EEA22EF50F60A02E18EEF1FF000
:1001E000030A02E163EF1FF0010A02E118EF1FF0BA
:1001F000070A02E1D7EF1EF0020A02E191EF1EF0BA
:10020000010A02E154EF1EF0020A02E137EF1EF08C
:10021000AB0A02E1D9EF1DF0010A02E17FEF1DF008
:100220000F0A02E14FEF1DF0010A02E1D0EF1CF0CE
:10023000030A02E153EF1CF0010A02E10CEF1CF08B
:10024000070A02E1DAEF1BF01B0A02E166EF1BF07E
:100250000F0A02E155EF1BF0010A02E149EF1BF022
:10026000030A02E10DEF1BF0010A02E12AEF19F087
:10027000070A02E109EF19F0010A02E1A0EF18F004
:10028000030A02E142EF18F0010A02E10DEF18F053
:100290007D0A02E1B9EF17F0010A02E171EF17F0F0
:1002A000070A02E166EF17F0010A02E1FDEF16F01E
:1002B000030A02E190EF16F0010A02E179EF16F06D
:1002C0000F0A02E141EF16F0080A02E191EF15F082
:1002D000760A02E118EF15F0770A02E1A7EF14F0B1
:1002E000080A02E142EF14F0030A02E1E2EF13F020
:1002F000010A02E167EF13F0070A02E1E1EF12F0F1
:10030000010A02E1A5EF12F0030A02E16AEF12F01E
:10031000010A02E12DEF12F01F0A02E1D8EF11F0FD
:10032000020A02E163EF11F0030A02E1C8EF10F0E4
:10033000020A02E121EF10F0070A02E1E9EF0FF0F3
:10034000010A02E196EF0FF0030A02E145EF0FF018
:10035000010A02E1C4EF0EF00F0A02E144EF0EF0D1
:10036000010A02E1E9EF0DF0030A02E1A2EF0DF04C
:10037000010A02E13CEF0DF0070A02E106EF0DF081
:10038000010A02E1D0EF0CF0030A02E183EF0CF066
:10039000730A02E12CEF0CF0030A02E1BDEF0BF04F
:1003A000010A02E137EF0BF0700A02E16CEF09F08D
:1003B0003F0A02E13AEF09F0010A02E116EF09F003
:1003C000030A02E1F1EF08F0010A02E1CDEF08F0C3
:1003D000070A02E1A8EF08F0010A02E182EF08F043
:1003E000030A02E15DEF08F0010A02E139EF08F0CB
:1003F0000F0A02E1E5EF07F0010A02E1C1EF07F0A1
:10040000030A02E15FEF07F0010A02E109EF07F0DA
:10041000070A02E190EF06F0010A02E123EF06F07D
:10042000030A01E1A5D3010A01E189D31F0A01E111
:100430000AD3010A01E1BBD2030A01E120D2010A79
:1004400001E1F9D1070A01E1C5D1010A01E1AAD10F
:10045000030A01E191D1010A01E178D10F0A01E11A
:10046000F7D0010A01E1E8D0030A01E1BFD0010A97
:1004700001E199D0070A65E0010A42E0030A0AE0B7
:10048000010A02E0CBEF1FF0E66ADDEC1FF0E55257
:10049000D0EF1FF0010EE66EDDEC1FF0E552D2DD6D
:1004A000E66ADDEC1FF0E5520C0EE66EDDEC1FF0A7
:1004B000E552E66ADDEC1FF0E552E66ADDEC1FF07E
:1004C000E552E66ADDEC1FF0E552010EE66EDDEC6A
:1004D0001FF0E552200EE66EDDEC1FF0E552520EE5
:1004E000E66EDDEC1FF0E552530EE66EDDEC1FF01C
:1004F000E552540EE66EDDEC1FF0E552D0EF1FF032
:10050000020EE66EDDEC1FF0E552E66ADDEC1FF050
:10051000E5520C0EE66EDDEC1FF0E552E66ADDEC0E
:100520001FF0E552E66ADDEC1FF0E552E66ADDEC0D
:100530001FF0E552010EE66EDDEC1FF0E552D0EF44
:100540001FF0030EE66EDDEC1FF0E55200282A6E68
:10055000010114512A5C18E2002A0050EA6AA00F37
:10056000E96E000EEA22EFCFDFFF590EDF5C06E2F4
:10057000DFCFE6FFDDEC1FF0E55205D0FE0EE66EA4
:10058000DDEC1FF0E5520DD0FE0EE66EDDEC1FF047
:10059000E5520028EA6AA00FE96E000EEA22040E76
:1005A000EF6ED0EF1FF0400E015C09E20150EA6AE5
:1005B000600FE96E000EEA22EF6A012AF4D7016AA1
:1005C00004010CBF0CD0400EE66E600EE66E000E0D
:1005D000E66E48EC21F0E552E552E55203D0000109
:1005E000010EEA6F14C100F0D0EF1FF0050EE66EA9
:1005F000DDEC1FF0E552000E036E046A096E0A6A14
:10060000076E086A840ECB6E040ECA6E0B0EBC6EAB
:10061000B80EBB6E9E9C9D8CB36AB26A890EB16E99
:100620000B0EBA6EBE6A0C0EBD6E9494C00EF26EC6
:100630001E0ED26ED0EF1FF0060EE66EDDEC1FF040
:10064000E5529D9CBA6ABD6A0E0ED26ED0EF1FF0C5
:10065000070EE66EDDEC1FF0E552030E00242A6E55
:10066000010114512A5C63E2002A0050EA6AA00FDB
:10067000E96E000EEA22EF500D6E0D50030A40E0C5
:10068000010A2BE0030A16E0010A01E04CD0002A1F
:100690000050EA6AA00FE96E000EEA22EF50066EE3
:1006A000002A0050EA6AA00FE96E000EEA22EFCF9E
:1006B000ECF03CD0002A0050EA6AA00FE96E000E70
:1006C000EA22EFCFF0F0002A0050EA6AA00FE96EAC
:1006D000000EEA22EFCFEFF029D0002A0050EA6A9C
:1006E000A00FE96E000EEA22EFCFF2F0002A0050D0
:1006F000EA6AA00FE96E000EEA22EFCFF1F016D001
:10070000002A0050EA6AA00FE96E000EEA22EFCF3D
:10071000EDF0002A0050EA6AA00FE96E000EEA220E
:10072000EFCFEEF003D0020E002600D00DD0FE0E6B
:10073000E66EDDEC1FF0E5520028EA6AA00FE96ED4
:10074000000EEA22040EEF6ED0EF1FF0080EE66EE8
:10075000DDEC1FF0E552F29E06500D6E0D5009E0E3
:1007600000000000000000000000000000000D0676
:10077000F5D7F28ED0EF1FF0090EE66EDDEC1FF01C
:10078000E552F29EECC00DF00D5009E000000000B3
:10079000000000000000000000000D06F5D7F28EFA
:1007A000D0EF1FF00A0EE66EDDEC1FF0E552F29E70
:1007B000EFC013F0F0C014F01350141008E0000064
:1007C0000000000000001306000E145AF5D7F28E48
:1007D000D0EF1FF00B0EE66EDDEC1FF0E5520028A7
:1007E0002A6E010114512A5C17E2F29E002A005081
:1007F000EA6AA00FE96E000EEA22EF500D6E0D506E
:1008000009E00000000000000000000000000000FF
:100810000D06F5D7F28E0DD0FE0EE66EDDEC1FF064
:10082000E5520028EA6AA00FE96E000EEA22040EE3
:10083000EF6ED0EF1FF0A1940C0EE66EDDEC1FF012
:10084000E552F29EC282C2B2FED79E9CF28EA1A455
:100850000AD0E66ADDEC1FF0E552E66ADDEC1FF037
:10086000E552D0EF1FF0C450E66EDDEC1FF0E5520C
:10087000C350E66EDDEC1FF0E552D0EF1FF00D0E19
:10088000E66EDDEC1FF0E55200282A6E01011451DE
:100890002A5C01E37DD09D50400B03E0D250200B39
:1008A00006E1FE0EE66EDDEC1FF0E55270D0A1947D
:1008B000002A0050EA6AA00FE96E000EEA22EF500B
:1008C000136E146A13C00BF014C00CF0480E0C0227
:1008D000F3CF0CF0480E0B02F3CF0BF0F4500C26C4
:1008E0000A0E276E286A0BC022F00CC023F0D0EC51
:1008F00026F022C00BF023C00CF00F0E0D6EE80E98
:10090000136E030E146E1350141008E00000000064
:10091000000000001306000E145AF5D70D06083427
:1009200004E207500E08000E085408E3D88008506F
:1009300004E7F20E075CFF0E085802E20D50DFE1FB
:10094000A1A405D0E66ADDEC1FF0E55220D0083402
:1009500004E207500E08000E085408E3D88008503F
:1009600004E7F20E075CFF0E085806E2FE0EE66E84
:10097000DDEC1FF0E5520BD00050EA6AA00FE96EE3
:10098000000EEA22EF50E66EDDEC1FF0E5520DD0CE
:10099000FE0EE66EDDEC1FF0E5520028EA6AA00FBD
:1009A000E96E000EEA22040EEF6ED0EF1FF00E0E7D
:1009B000E66EDDEC1FF0E55200282A6E01011451AD
:1009C0002A5C32E2002A0050EA6AA00FE96E000EAB
:1009D000EA22EF500D6E010E0D1402E0000E01D060
:1009E000010EE8B08B82E8A08B92020E0D1402E09B
:1009F000010E01D0000EE8B09482E8A09492040E9B
:100A00000D1402E0010E01D0000EE8B08B80E8A0CA
:100A10008B90080E0D1402E0010E01D0000EE8B01C
:100A20009480E8A094900DD0FE0EE66EDDEC1FF0F1
:100A3000E5520028EA6AA00FE96E000EEA22040ED1
:100A4000EF6ED0EF1FF00F0EE66EDDEC1FF0E552FB
:100A500000282A6E010114512A5C62E2002A00502B
:100A6000EA6AA00FE96E000EEA22EF50010B02E0E5
:100A7000010E01D0000EE8B08A8AE8A08A9A0050E0
:100A8000EA6AA00FE96E000EEA22EF50020B02E0C4
:100A9000010E01D0000EE8B0938AE8A0939A0050AE
:100AA000EA6AA00FE96E000EEA22EF50040B02E0A2
:100AB000010E01D0000EE8B08A8CE8A08A9C00509C
:100AC000EA6AA00FE96E000EEA22EF50080B02E07E
:100AD000010E01D0000EE8B0938CE8A0939C00506A
:100AE000EA6AA00FE96E000EEA22EF50100B02E056
:100AF000010E01D0000EE8B08A8EE8A08A9E005058
:100B0000EA6AA00FE96E000EEA22EF50200B02E025
:100B1000010E01D0000EE8B0938EE8A0939E0DD098
:100B2000FE0EE66EDDEC1FF0E5520028EA6AA00F2B
:100B3000E96E000EEA22040EEF6ED0EF1FF0100EE9
:100B4000E66EDDEC1FF0E5520D6A81BA0D8093BAB6
:100B50000D8281BC0D8493BC0D8681BE0D8893BE31
:100B60000D8A0D50E66EDDEC1FF0E552D0EF1FF060
:100B7000110EE66EDDEC1FF0E552020E00242A6E27
:100B8000010114512A5C50E2002A0050EA6AA00FC9
:100B9000E96E000EEA22EFCF14F0002A0050EA6A54
:100BA000A00FE96E000EEA22EFCF13F0F29E8A9AB0
:100BB0008A8C00008A9C00008A8C00008A9C0000BD
:100BC0008A8C00008A9C00008A8C00008A9C0000AD
:100BD0008A8C00008A9C00008A8C00008A9C00009D
:100BE00006500D6E0D5009E00000000000000000EE
:100BF0000000000000000D06F5D78A8C00008A9CDA
:100C000000000E0E0D6E143213328A9AD8B08A8A02
:100C10008A8C00008A9C0D2EF6D78A9A8A8C000056
:100C20008A9C0000F28E0DD0FE0EE66EDDEC1FF009
:100C3000E5520028EA6AA00FE96E000EEA22040ECF
:100C4000EF6ED0EF1FF0120EE66EDDEC1FF0E552F6
:100C5000020E00242A6E010114512A5C52E2002A7D
:100C60000050EA6AA00FE96E000EEA22EFCF14F0FE
:100C7000002A0050EA6AA00FE96E000EEA22EFCFC8
:100C800013F0F29E8A9A8A8C00008A9C00008A8A5D
:100C90008A8C00008A9C00008A9A8A8C00008A9CB8
:100CA00000008A8C00008A9C00008A8C00008A9CCC
:100CB00000008A8C00008A9C000006500D6E0D50CA
:100CC00009E000000000000000000000000000003B
:100CD0000D06F5D78A8C00008A9C00000E0E0D6E62
:100CE000143213328A9AD8B08A8A8A8C00008A9C7D
:100CF0000D2EF6D78A9A8A8C00008A9C0000F28E0C
:100D00000DD0FE0EE66EDDEC1FF0E5520028EA6A1B
:100D1000A00FE96E000EEA22040EEF6ED0EF1FF076
:100D2000130EE66EDDEC1FF0E55200282A6E01017D
:100D300014512A5C5FE2002A0050EA6AA00FE96EB3
:100D4000000EEA22EFCF13F0F29E8A8A8A8C00000E
:100D50008A9C00008A8C00008A9C00008A9A8A8CF7
:100D600000008A9C00008A8C00008A9C00008A8C0B
:100D700000008A9C00008A8C00008A9C00000650BB
:100D80000D6E0D5009E000000000000000000000A2
:100D9000000000000D06F5D78A8C00008A9C000038
:100DA000080E0D6E13328A9AD8B08A8A8A8C000097
:100DB0008A9C0D2EF7D78A9A8A8C00008A9C0000A4
:100DC0008A8C00008A9C00008A8C00008A9C0000AB
:100DD0008A8C00008A9C00008A8C00008A9C00009B
:100DE0008A8C00008A9C00008A8C00008A9C00008B
:100DF000F28E0DD0FE0EE66EDDEC1FF0E5520028FF
:100E0000EA6AA00FE96E000EEA22040EEF6ED0EF40
:100E10001FF0140EE66EDDEC1FF0E552F29E8A9A8A
:100E20008A8C00008A9C00008A8C00008A9C00004A
:100E30008A8A8A8C00008A9C00008A9A8A8C000028
:100E40008A9C00008A8C00008A9C00008A8C00002A
:100E50008A9C0000938A06500D6E0D5009E0000038
:100E60000000000000000000000000000D06F5D7A3
:100E70008A8C00008A9C00000E0E0D6E8A8C000089
:100E80008A9CD8908A9C81BAD880143213320D2E55
:100E9000F5D7D89014321332D890143213328A8C8A
:100EA000939A8A9CF28E14C0E6FFDDEC1FF0E552A7
:100EB00013C0E6FFDDEC1FF0E552D0EF1FF0150E7A
:100EC000E66EDDEC1FF0E552F29E8A8A8A8C000005
:100ED0008A9C00008A9A8A8C00008A9C00008A8A78
:100EE0008A8C00008A9C00008A9A8A8C00008A9C66
:100EF00000008A8C00008A9C00008A8C00008A9C7A
:100F00000000938A06500D6E0D5009E000000000AD
:100F1000000000000000000000000D06F5D78A8CDC
:100F200000008A9C0000080E0D6E8A8C00008A9CCE
:100F3000D89081BAD88013320D2EF7D78A8C000052
:100F40008A9C00008A8C00008A9C00008A8C000029
:100F50008A9C00008A8C00008A9C00008A8C000019
:100F60008A9C00008A8C00008A9C00008A8C939ADC
:100F70008A9CF28E13C0E6FFDDEC1FF0E552D0EF45
:100F80001FF0160EE66EDDEC1FF0E552F29E8A9A17
:100F90008A8C00008A9C00008A8A8A8C00008A9CC5
:100FA00000008A8C00008A9C00008A9A8A8C0000CB
:100FB0008A9C00008A8C00008A9C00008A8C0000B9
:100FC0008A9C0000F28ED0EF1FF0170EE66EDDEC6B
:100FD0001FF0E55200282A6E010114512A5C3AE202
:100FE000F29E002A0050EA6AA00FE96E000EEA2283
:100FF000EFCF13F0000113502BE08A9A8A8C000087
:101000008A9C00008A8A8A8C00008A9C00008A8C54
:1010100000008A9C00008A9A8A8C00008A9C00004A
:101020008A8C00008A9C00008A8C00008A9C000048
:1010300006500D6E0D5009E0000000000000000099
:101040000000000000000D06F5D700011306D2D7FE
:10105000F28E0DD0FE0EE66EDDEC1FF0E55200289C
:10106000EA6AA00FE96E000EEA22040EEF6ED0EFDE
:101070001FF0180EE66EDDEC1FF0E552F29E8A9A24
:101080008A8C00008A9C00008A8C00008A9C0000E8
:101090008A8C00008A9C00008A8A8A8C00008A9CC4
:1010A00000008A9A8A8C00008A9C00008A8C0000CA
:1010B0008A9C0000F28ED0EF1FF0190EE66EDDEC78
:1010C0001FF0E552F29E8A8A8A8C00008A9C0000FA
:1010D0008A9A8A8C00008A9C00008A8C00008A9C74
:1010E00000008A8A8A8C00008A9C00008A9A8A8C76
:1010F00000008A9C00008A8C00008A9C0000F28E0E
:10110000D0EF1FF01A0EE66EDDEC1FF0E552F29EF6
:101110008A9A8A8C00008A9C00008A8A8A8C000045
:101120008A9C00008A9A8A8C00008A9C00008A8A25
:101130008A8C00008A9C00008A9A8A8C00008A9C13
:1011400000008A8C00008A9C0000F28ED0EF1FF015
:101150001B0EE66EDDEC1FF0E552F29E8A8A8A8C49
:1011600000008A9C00008A8C00008A9C00008A9AF9
:101170008A8C00008A9C00008A8A8A8C00008A9CE3
:1011800000008A9A8A8C00008A9C00008A8C0000E9
:101190008A9C0000F28ED0EF1FF01C0EE66EDDEC94
:1011A0001FF0E552F29E8A9A8A8C00008A9C000009
:1011B0008A8A8A8C00008A9C00008A8C00008A9CA3
:1011C00000008A8C00008A9C00008A9A8A8C0000A9
:1011D0008A9C00008A8C00008A9C0000F28ED0EF6E
:1011E0001FF01D0EE66EDDEC1FF0E552F29E8A8ABE
:1011F0008A8C00008A9C00008A9A8A8C00008A9C53
:1012000000008A8C00008A9C00008A8C00008A9C66
:1012100000008A8A8A8C00008A9C00008A9A8A8C44
:1012200000008A9C0000F28ED0EF1FF01E0EE66ECA
:10123000DDEC1FF0E552F29E8A9A8A8C00008A9CAF
:1012400000008A8C00008A9C00008A8C00008A9C26
:1012500000008A8A8A8C00008A9C00008A8C000028
:101260008A9C00008A9A8A8C00008A9C0000F28E78
:10127000D0EF1FF01F0EE66EDDEC1FF0E5520028E8
:101280002A6E010114512A5C18E2002A0050EA6A11
:10129000A00FE96E000EEA22EFCF13F0F29E060EC9
:1012A0000D6E13328A9AD8B08A8A8A8C00008A9C82
:1012B0000D2EF7D78A9AF28E0DD0FE0EE66EDDEC7B
:1012C0001FF0E5520028EA6AA00FE96E000EEA223C
:1012D000040EEF6ED0EF1FF0200EE66EDDEC1FF077
:1012E000E552020E00242A6E010114512A5C01E32A
:1012F000AFD1002A0050EA6AA00FE96E000EEA2280
:10130000EFCF14F0002A0050EA6AA00FE96E000E39
:10131000EA22EFCF13F0010E13C0DBFF020E14C060
:10132000DBFFF29E8A9A8A8C00008A9C00008A8ADF
:101330008A8C00008A9C00008A9A8A8C00008A9C11
:1013400000008A8C00008A9C00008A8C00008A9C25
:1013500000008A8C00008A9C000006500D6E0D5023
:1013600009E0000000000000000000000000000094
:101370000D06F5D78A8C00008A9C00000E0E0D6EBB
:10138000143213328A9AD8B08A8A8A8C00008A9CD6
:101390000D2EF6D78A9A8A8C00008A9C0000030ED4
:1013A000DB6A040EDB6A030EDBCF2AF0040EDBCF10
:1013B0002BF00001ED5100012BAE02D0D89003D0EC
:1013C0002A5C000E2B5801E3BED08A9A8A8C00005A
:1013D0008A9C00008A8C00008A9C00008A8C000095
:1013E0008A9C00008A8A8A8C00008A9C00008A9A63
:1013F0008A8C00008A9C00008A8C00008A9C000075
:10140000ECC00DF00D5009E00000000000000000ED
:101410000000000000000D06F5D78A9A8A8C0000B3
:101420008A9C00008A8A8A8C00008A9C00008A8C30
:1014300000008A9C00008A8C00008A9C00008A9A26
:101440008A8C00008A9C00008A8C00008A9C000024
:1014500006500D6E0D5009E0000000000000000075
:101460000000000000000D06F5D78A9A8A8C000063
:101470008A9C00008A8C00008A9C00008A8A8A8CE0
:1014800000008A9C00008A9A8A8C00008A9C0000D6
:101490008A8C00008A9C00008A8C00008A9C0000D4
:1014A000938A06500D6E0D5009E000000000000008
:1014B00000000000000000000D06F5D78A8C000037
:1014C0008A9C00000E0E0D6E8A8C00008A9CD890BB
:1014D00081BAD880143213320D2EF6D7D890143238
:1014E0001332D890143213328A8C939A8A9C065005
:1014F0000D6E0D5009E0000000000000000000002B
:10150000000000000D06F5D7010EDBCF2AF0020E19
:10151000DBCF2BF013502A1802E114502B180DE1E9
:10152000030EDBCF2AF0040EDBCF2BF0010E2A24B2
:101530000D6E030EDB68040EDB6A030EDB2A040E5D
:1015400001E3DB2A30D7F28EF29ED950030FE96E09
:10155000DACFEAFFEE5002E1010EED1872E10D5014
:10156000E66EDDEC1FF0E5520001EE510D02F35086
:10157000E66ED950030FE96EDACFEAFFE552E75085
:10158000EE6EED6AD950030FE96EDACFEAFFEE5046
:10159000ED1056E08A9A8A8C00008A9C00008A8CA2
:1015A00000008A9C00008A8C00008A9C00008A8AC5
:1015B0008A8C00008A9C00008A9A8A8C00008A9C8F
:1015C00000008A8C00008A9C0000ECC00DF00D50D9
:1015D00009E0000000000000000000000000000022
:1015E0000D06F5D78A9A8A8C00008A9C00008A8AA8
:1015F0008A8C00008A9C00008A8C00008A9C000073
:101600008A8C00008A9C00008A9A8A8C00008A9C3E
:1016100000008A8C00008A9C000006500D6E0D5060
:1016200009E00000000000000000000000000000D1
:101630000D06F5D7030EDB06040E01E2DB06A2D78A
:1016400005D0FE0EE66EDDEC1FF0E552F28E0DD0F9
:10165000FE0EE66EDDEC1FF0E5520028EA6AA00FF0
:10166000E96E000EEA22040EEF6ED0EF1FF0500E6E
:10167000E66EDDEC1FF0E552020E00242A6E010139
:1016800014512A5C6BE2002A0050EA6AA00FE96E4E
:10169000000EEA22EFCF14F0002A0050EA6AA00FF1
:1016A000E96E000EEA22EFCF13F0F29E8A8A8A8C4E
:1016B00000008A9C00008A9A8A8C00008A9C0000A4
:1016C0008A8A8A8C00008A9C00008A8C00008A9C8E
:1016D00000008A8C00008A9C00008A9A8A8C000094
:1016E0008A9C000006500D6E0D5009E000000000BD
:1016F000000000000000000000000D06F5D78A8CF5
:1017000000008A9C0000100E0D6E143213328A9A6B
:10171000D8B08A8A8A8C00008A9C0D2EF6D78A9AC5
:101720008A8C00008A9C00008A8C00008A9C000041
:101730008A8C00008A9C00008A8C00008A9C000031
:101740008A8C00008A9C00008A8C00008A9C000021
:101750008A8C00008A9C0000F28E0DD0FE0EE66E90
:10176000DDEC1FF0E5520028EA6AA00FE96E000EDA
:10177000EA22040EEF6ED0EF1FF0510EE66EDDECA4
:101780001FF0E552020E00242A6E010114512A5C5A
:1017900054E2002A0050EA6AA00FE96E000EEA2225
:1017A000EFCF14F0002A0050EA6AA00FE96E000E95
:1017B000EA22EFCF13F0F29E8A9A8A8C00008A9C6C
:1017C00000008A8A8A8C00008A9C00008A9A8A8C8F
:1017D00000008A9C00008A8C00008A9C00008A8C91
:1017E00000008A9C00008A8A8A8C00008A9C000083
:1017F00006500D6E0D5009E00000000000000000D2
:101800000000000000000D06F5D78A9A8A8C0000BF
:101810008A9C00000E0E0D6E143213328A9AD8B0D4
:101820008A8A8A8C00008A9C0D2EF6D78A9A8A8C26
:1018300000008A9C0000F28E0DD0FE0EE66EDDECFC
:101840001FF0E5520028EA6AA00FE96E000EEA22B6
:10185000040EEF6ED0EF1FF0520EE66EDDEC1FF0BF
:10186000E552F29E8A9A8A8C00008A9C00008A8C3B
:1018700000008A9C00008A8A8A8C00008A9C0000F2
:101880008A9A8A8C00008A9C00008A8C00008A9CBC
:1018900000008A8A8A8C00008A9C0000938A065085
:1018A0000D6E0D5009E00000000000000000000077
:1018B000000000000D06F5D78A9A8A8C00008A9CE9
:1018C00000000E0E0D6E8A8C00008A9CD89081BAA2
:1018D000D880143213320D2EF6D7D890143213322A
:1018E000D890143213328A8C939A8A9CF28E14C048
:1018F000E6FFDDEC1FF0E55213C0E6FFDDEC1FF064
:10190000E552D0EF1FF0210EE66EDDEC1FF0E55240
:10191000020E00242A6E010114512A5C32E2F29E6A
:101920008A8C939A8A9A8A9C8A8C00008A9C0000EE
:101930008A8C00008A9C00008A8C00008A9C00002F
:10194000002A0050EA6AA00FE96E000EEA22EFCFEB
:1019500014F0002A0050EA6AA00FE96E000EEA2295
:10196000EFCF13F0100E0D6E143213328A9AD8B0E6
:101970008A8A8A8C00008A9C0D2EF6D78A9AF28E6B
:101980000DD0FE0EE66EDDEC1FF0E5520028EA6A8F
:10199000A00FE96E000EEA22040EEF6ED0EF1FF0EA
:1019A000220EE66EDDEC1FF0E552F29E8A8C939AD1
:1019B0008A9A8A9C8A8A8A8C8A9C8A9A8A8C8A9C2D
:1019C0008A8C8A9C8A8C8A9C8A8C8A9C8A8C8A9C27
:1019D0008A8C8A9C8A8C8A9C8A8C8A9C8A8C8A9C17
:1019E0008A8C8A9C938A080E0D6E8A8C8A9CD89069
:1019F00081BAD88013320D2EF8D78A9AF28E13C08E
:101A0000E6FFDDEC1FF0E552D0EF1FF0230EE66E8F
:101A1000DDEC1FF0E552F29E8A8C939A8A9A8A9C9A
:101A20008A8C8A9C8A8C8A9C8A8A8A8C8A9C8A9ACA
:101A30008A8C8A9C8A8C8A9C8A8C8A9C8A8C8A9CB6
:101A40008A8C8A9C8A8C8A9C8A8C8A9C8A8C8A9CA6
:101A5000938A080E0D6E8A8C8A9CD89081BAD880A1
:101A600013320D2EF8D78A9AF28E13C0E6FFDDEC02
:101A70001FF0E552D0EF1FF0240EE66EDDEC1FF0F4
:101A8000E552002A0050EA6AA00FE96E000EEA2231
:101A9000EF500D6E01011451005C45E201500D2420
:101AA0002A6E400E2A5C3FE20D50E66EDDEC1FF020
:101AB000E552050E0DC0DBFF050EDB5033E0F29E54
:101AC0008A8C939A8A8A8A9C8A9A8A8C8A9C8A8C23
:101AD0008A9C8A8A8A8C8A9C8A9A8A8C8A9C8A8C1A
:101AE0008A9C8A8C8A9C8A8C8A9C8A8C8A9C8A8C06
:101AF0008A9C8A8C8A9C8A8C8A9C938A080E0D6E9A
:101B00008A8C8A9CD89081BAD88013320D2EF8D74F
:101B10008A9AF28E13C0E6FFDDEC1FF0E552050E47
:101B2000DB06CAD70DD0FE0EE66EDDEC1FF0E552E7
:101B30000028EA6AA00FE96E000EEA22040EEF6E9A
:101B4000D0EF1FF0250EE66EDDEC1FF0E552020E21
:101B500000242A6E010114512A5C2CE2F29E8A8C28
:101B6000939A8A9A8A9C8A8C8A9C8A8A8A8C8A9C72
:101B70008A8C8A9C002A0050EA6AA00FE96E000E47
:101B8000EA22EFCF14F0002A0050EA6AA00FE96EB3
:101B9000000EEA22EFCF13F0100E0D6E1432133246
:101BA0008A9AD8B08A8A8A8C8A9C0D2EF7D78A9A0C
:101BB000F28E0DD0FE0EE66EDDEC1FF0E552002831
:101BC000EA6AA00FE96E000EEA22040EEF6ED0EF73
:101BD0001FF0260EE66EDDEC1FF0E552002A0050E5
:101BE000EA6AA00FE96E000EEA22EF500D6E005077
:101BF0000D240D242A6E010114512A5C36E2060ED2
:101C00000DC0DBFF060EDB502FE0F29E8A8C939A0C
:101C10008A8A8A9C8A9A8A8C8A9C8A8A8A8C8A9CDA
:101C20008A8C8A9C002A0050EA6AA00FE96E000E96
:101C3000EA22EFCF14F0002A0050EA6AA00FE96E02
:101C4000000EEA22EFCF13F0100E0D6E1432133295
:101C50008A9AD8B08A8A8A8C8A9C0D2EF7D78A9A5B
:101C6000F28E060EDB06CED70DD0FE0EE66EDDEC54
:101C70001FF0E5520028EA6AA00FE96E000EEA2282
:101C8000040EEF6ED0EF1FF0270EE66EDDEC1FF0B6
:101C9000E552040E00242A6E010114512A5C65E20B
:101CA000F29E8A8C939A8A8A8A9C8A8C8A9C8A8CD5
:101CB0008A9C8A8C8A9C002A0050EA6AA00FE96EEE
:101CC000000EEA22EFCF14F0002A0050EA6AA00FBB
:101CD000E96E000EEA22EFCF13F0100E0D6E1432F3
:101CE00013328A9AD8B08A8A8A8C8A9C0D2EF7D7AA
:101CF0008A9A8A8C8A9C8A8C8A9C8A8C8A9C8A8CF6
:101D0000002A0050EA6AA00FE96E000EEA22EFCF27
:101D100014F0002A0050EA6AA00FE96E000EEA22D1
:101D2000EFCF13F01350141008E000000000000083
:101D300000001306000E145AF5D78A9CECC00DF073
:101D40000D5009E00000000000000000000000004D
:101D500000000D06F5D7100E0D6E0D5004E08A8CB4
:101D60008A9C0D06FAD7F28E0DD0FE0EE66EDDECE3
:101D70001FF0E5520028EA6AA00FE96E000EEA2281
:101D8000040EEF6ED0EF1FF0280EE66EDDEC1FF0B4
:101D9000E552040E00242A6E010114512A5C66E209
:101DA000F29E8A8C939A8A9A8A9C8A8A8A8C8A9CC6
:101DB0008A8C8A9C8A8C8A9C002A0050EA6AA00F2E
:101DC000E96E000EEA22EFCF14F0002A0050EA6A12
:101DD000A00FE96E000EEA22EFCF13F0100E0D6E89
:101DE000143213328A9AD8B08A8A8A8C8A9C0D2E31
:101DF000F7D78A9A8A8C8A9C8A8C8A9C8A8C8A9C3D
:101E00008A8C002A0050EA6AA00FE96E000EEA22CE
:101E1000EFCF14F0002A0050EA6AA00FE96E000E1E
:101E2000EA22EFCF13F01350141008E00000000076
:101E3000000000001306000E145AF5D78A9CECC06F
:101E40000DF00D5009E0000000000000000000004F
:101E5000000000000D06F5D7100E0D6E0D5004E0C9
:101E60008A8C8A9C0D06FAD7F28E0DD0FE0EE66E95
:101E7000DDEC1FF0E5520028EA6AA00FE96E000EC3
:101E8000EA22040EEF6ED0EF1FF0290EE66EDDECB5
:101E90001FF0E552030E00242A6E010114512A5C42
:101EA00036E2002A0050EA6AA00FE96E000EEA222C
:101EB000EFCF13F0F29E8A8C939A040E0D6E1332BC
:101EC0008A9AD8B08A8A8A8C8A9C0D2EF8D7002AE2
:101ED0000050EA6AA00FE96E000EEA22EFCF14F07C
:101EE000002A0050EA6AA00FE96E000EEA22EFCF46
:101EF00013F0100E0D6E143213328A9AD8B08A8AFB
:101F00008A8C8A9C0D2EF7D78A9AF28E0DD0FE0EFF
:101F1000E66EDDEC1FF0E5520028EA6AA00FE96EDC
:101F2000000EEA22040EEF6ED0EF1FF02A0EE66ECE
:101F3000DDEC1FF0E55200282A6E010114512A5CE5
:101F400039E2002A0050EA6AA00FE96E000EEA2288
:101F5000EFCF13F0F29E8A8C939A040E0D6E13321B
:101F60008A9AD8B08A8A8A8C8A9C0D2EF8D78A8C55
:101F70008A9C8A8C8A9C8A8C8A9C8A8C8A9C8A8C71
:101F80008A9C8A8C8A9C8A8C8A9C8A8C8A9C938A5A
:101F9000080E0D6E8A8C8A9CD89081BAD880133234
:101FA0000D2EF8D78A9AF28E13C0E6FFDDEC1FF0F3
:101FB000E5520DD0FE0EE66EDDEC1FF0E552002876
:101FC000EA6AA00FE96E000EEA22040EEF6ED0EF6F
:101FD0001FF02B0EE66EDDEC1FF0E55200282A6E96
:101FE000010114512A5C1EE2002A0050EA6AA00F87
:101FF000E96E000EEA22EF500D6EFF0E0D5C03E15C
:102000009368948C0ED0C70E936E8A6A0DB08A8640
:102010000DB28A880DB48A8A949C8B9C0001050EAF
:10202000EC6F0DD0FE0EE66EDDEC1FF0E5520028E1
:10203000EA6AA00FE96E000EEA22040EEF6ED0EFFE
:102040001FF02C0EE66EDDEC1FF0E552030E0024AF
:102050002A6E010114512A5C01E38BD0002A005042
:10206000EA6AA00FE96E000EEA22EF500D6E000141
:10207000010E146E002A0050EA6AA00FE96E000EED
:10208000EA22EFCF13F09BEC20F00D5042E0FE0E61
:1020900000011314E66EBDEC20F0E5529FEC20F039
:1020A000000936E1002A0050EA6AA00FE96E000E2E
:1020B000EA22EF50E66EBDEC20F0E5529FEC20F0F6
:1020C000000926E1DFEC20F0010E00011310E66E9E
:1020D000BDEC20F0E5529FEC20F0000919E1000171
:1020E000146A0D50E66EDDEC1FF0E5520D500EE067
:1020F000A8EC20F0F350E66EDDEC1FF0E5520D5039
:10210000010802E2FAEC20F00D06F0D7F4EC20F022
:1021100019D0010E00011310E66EBDEC20F0E5525F
:102120009FEC20F000090EE1010EE66EDDEC1FF0E1
:10213000E552A8EC20F0F350E66EDDEC1FF0E5521E
:10214000F4EC20F09FEC20F0000910E000011450A6
:102150000DE0FD0EE66EDDEC1FF0E5520028EA6AA8
:10216000A00FE96E000EEA22040EEF6EE9EC20F0FB
:102170000DD0FE0EE66EDDEC1FF0E5520028EA6A97
:10218000A00FE96E000EEA22040EEF6ED0EF1FF0F2
:102190002E0EE66EDDEC1FF0E552040E00242A6ED2
:1021A000010114512A5C01E37FD0002A0050EA6A41
:1021B000A00FE96E000EEA22EF500D6E0001010E35
:1021C000146E002A0050EA6AA00FE96E000EEA229F
:1021D000EFCF13F09BEC20F0FE0E00011314E66E1F
:1021E000BDEC20F0E5529FEC20F0000946E1002A0A
:1021F0000050EA6AA00FE96E000EEA22EF50E66E88
:10220000BDEC20F0E5529FEC20F0000936E1002AF9
:102210000050EA6AA00FE96E000EEA22EF50E66E67
:10222000BDEC20F0E5529FEC20F0000926E1DFEC48
:1022300020F0010E00011310E66EBDEC20F0E55217
:102240009FEC20F0000919E10001146A0D50E66EC0
:10225000DDEC1FF0E5520D500EE0A8EC20F0F3503D
:10226000E66EDDEC1FF0E5520D50010802E2FAECDB
:1022700020F00D06F0D7F4EC20F09FEC20F00009E0
:1022800010E0000114500DE0FD0EE66EDDEC1FF0D5
:10229000E5520028EA6AA00FE96E000EEA22040E59
:1022A000EF6EE9EC20F00DD0FE0EE66EDDEC1FF0D7
:1022B000E5520028EA6AA00FE96E000EEA22040E39
:1022C000EF6ED0EF1FF02D0EE66EDDEC1FF0E55245
:1022D000002A0050EA6AA00FE96E000EEA22EF50D1
:1022E0000D6E020E00240D242A6E010114512A5C89
:1022F00050E29BEC20F0002A0050EA6AA00FE96E41
:10230000000EEA22EF50FE0BE66EBDEC20F0E55227
:102310009FEC20F000092BE1002A0050EA6AA00F90
:10232000E96E000EEA22EF50E66EBDEC20F0E552B9
:102330009FEC20F000091BE10D50E66EDDEC1FF074
:10234000E5520D5014E0002A0050EA6AA00FE96E31
:10235000000EEA22EF50E66EBDEC20F0E5529FEC55
:1023600020F0000902E00D6802D00D06EAD70D50FA
:102370000DE0FD0EE66EDDEC1FF0E5520028EA6A86
:10238000A00FE96E000EEA22040EEF6EE9EC20F0D9
:102390000DD0FE0EE66EDDEC1FF0E5520028EA6A75
:1023A000A00FE96E000EEA22040EEF6ED0EF1FF0D0
:1023B0002F0EE66EDDEC1FF0E55200282A6E0101BB
:1023C00014512A5C3BE2002A0050EA6AA00FE96E31
:1023D000000EEA22EF500D6EFF0E0D5C09E19368CE
:1023E000948C948E010E066E0001640EEC6F25D065
:1023F000E50E936E0DA602D08A8201D08A92949C3B
:102400008B9C949E0C0E0D140001EC6F030E0D16A8
:102410000D5003E1120E066E10D00D0403E1080EFC
:10242000066E0BD0020E0D5C03E1050E066E05D0A4
:10243000030E0D5C02E1020E066E0DD0FE0EE66E7E
:10244000DDEC1FF0E5520028EA6AA00FE96E000EED
:10245000EA22040EEF6ED0EF1FF0300EE66EDDECD8
:102460001FF0E55200282A6E010114512A5C23E274
:10247000002A0050EA6AA00FE96E000EEA22EF502F
:102480000D6E0D50E66EDDEC1FF0E5520D5005E1CE
:10249000E66ADDEC1FF0E5520DD093800D500AE0A6
:1024A000E66A10EC21F0E552E66EDDEC1FF0E55235
:1024B0000D06F4D70DD0FE0EE66EDDEC1FF0E552F2
:1024C0000028EA6AA00FE96E000EEA22040EEF6E01
:1024D000D0EF1FF0310EE66EDDEC1FF0E552002A62
:1024E0000050EA6AA00FE96E000EEA22EF500D6E6E
:1024F00000500D242A6E010114512A5C17E20D5080
:10250000E66EDDEC1FF0E552949E0D500EE0002AC1
:102510000050EA6AA00FE96E000EEA22EF50E66E64
:1025200010EC21F0E5520D06F0D70DD0FE0EE66E50
:10253000DDEC1FF0E5520028EA6AA00FE96E000EFC
:10254000EA22040EEF6ED0EF1FF0320EE66EDDECE5
:102550001FF0E552020E00242A6E010114512A5C7C
:1025600021E2002A0050EA6AA00FE96E000EEA227A
:10257000EF508A6E002A0050EA6AA00FE96E000E42
:10258000EA22EF500D6EC00E0D142A6E3F0E8B1412
:102590002A108B6E380E0D142A6EC70E89142A105D
:1025A000896E0DD0FE0EE66EDDEC1FF0E5520028C0
:1025B000EA6AA00FE96E000EEA22040EEF6ED0EF79
:1025C0001FF0330EE66EDDEC1FF0E552030E002423
:1025D0002A6E010114512A5C6BE2002A0050EA6A5B
:1025E000A00FE96E000EEA22EF500D6E002A005097
:1025F000EA6AA00FE96E000EEA22EFCF14F0002A7B
:102600000050EA6AA00FE96E000EEA22EFCF13F045
:1026100001500D240D242A6E400E2A5C3BE20D5021
:10262000E66EDDEC1FF0E5520D5033E0200EE66E55
:1026300010EC21F0E55214C0E6FF10EC21F0E55259
:1026400013C0E6FF10EC21F0E552E66A10EC21F031
:10265000E552E66EDDEC1FF0E552280EE66E10EC5A
:1026600021F0E55214C0E6FF10EC21F0E55213C052
:10267000E6FF10EC21F0E552E66A10EC21F0E5529D
:10268000E66EDDEC1FF0E552132A000E14220D0653
:10269000CBD70DD0FE0EE66EDDEC1FF0E552002824
:1026A000EA6AA00FE96E000EEA22040EEF6E0DD06A
:1026B000FE0EE66EDDEC1FF0E5520028EA6AA00F80
:1026C000E96E000EEA22040EEF6ED0EF1FF0340E1A
:1026D000E66EDDEC1FF0E552002A0050EA6AA00F1A
:1026E000E96E000EEA22EF500D6E00500D240D240D
:1026F000020F2A6E010114512A5C55E20D50E66E5C
:10270000DDEC1FF0E552002A0050EA6AA00FE96EE6
:10271000000EEA22EFCF14F0002A0050EA6AA00F60
:10272000E96E000EEA22EFCF13F00D503BE0400EB1
:10273000E66E10EC21F0E55214C0E6FF10EC21F03B
:10274000E55213C0E6FF10EC21F0E552002A0050DC
:10275000EA6AA00FE96E000EEA22EF50E66E10EC76
:1027600021F0E552480EE66E10EC21F0E55214C05F
:10277000E6FF10EC21F0E55213C0E6FF10EC21F06B
:10278000E552002A0050EA6AA00FE96E000EEA2224
:10279000EF50E66E10EC21F0E552132A000E1422E1
:1027A0000D06C3D70DD0FE0EE66EDDEC1FF0E55230
:1027B0000028EA6AA00FE96E000EEA22040EEF6E0E
:1027C000D0EF1FF0350EE66EDDEC1FF0E55200286D
:1027D0002A6E010114512A5C46E2002A0050EA6A7E
:1027E000A00FE96E000EEA22EF500D6EFF0E0D5C99
:1027F00005E1BA6ABD6A8A96B16A34D09484939628
:10280000B368B26AC10EB16EBC6ABF6A0D5003E113
:102810003B0EBE6E21D00D0403E11D0EBE6E1CD01A
:10282000020E0D5C03E10B0EBE6E16D0030E0D5CA6
:1028300003E1050EBE6E10D0040E0D5C03E1020E26
:10284000BE6E0AD0050E0D5C03E1010EBE6E04D013
:10285000060E0D5C01E1BE6A010EBB6E0B0EBD6E75
:10286000020EBA6E0DD0FE0EE66EDDEC1FF0E552E4
:102870000028EA6AA00FE96E000EEA22040EEF6E4D
:10288000D0EF1FF0360EE66EDDEC1FF0E552030EC2
:1028900000242A6E010114512A5C4AE2F29E939AA6
:1028A0008A9A00008A8C0000000000008A9C0000C8
:1028B0008A8C0000000000008A9C00008A8C0000C6
:1028C000000000008A9C00008A8C000000000000CC
:1028D0008A9C002A0050EA6AA00FE96E000EEA22E4
:1028E000EFCF14F0002A0050EA6AA00FE96E000E44
:1028F000EA22EFCF13F0002A0050EA6AA00FE96E37
:10290000000EEA22EF500E6E180E0D6E14321332C6
:102910000E32D8A08A9AD8B08A8A00008A8C000029
:10292000000000008A9C0D2EF1D78A9AF28E0DD0FD
:10293000FE0EE66EDDEC1FF0E5520028EA6AA00FFD
:10294000E96E000EEA22040EEF6ED0EF1FF03E0E8D
:10295000E66EDDEC1FF0E552030E00242A6E010145
:1029600014512A5C56E2F29E939A8A9A00008A8C4D
:102970000000000000008A9C00008A8C000000001B
:1029800000008A9C00008A8C0000000000008A9CE5
:1029900000008A8C0000000000008A9C002A005081
:1029A000EA6AA00FE96E000EEA22EFCF14F0002AC7
:1029B0000050EA6AA00FE96E000EEA22EFCF13F092
:1029C000002A0050EA6AA00FE96E000EEA22EF50DA
:1029D0000E6E180E0D6E143213320E32D8A08A9A73
:1029E000D8B08A8A00008A8C0000000000008A9C0F
:1029F0000D2EF1D78A9A0D6A380E0D5C08E20000A0
:102A00008A8C0000000000008A9C0D2AF5D7F28E07
:102A10000DD0FE0EE66EDDEC1FF0E5520028EA6AEE
:102A2000A00FE96E000EEA22040EEF6ED0EF1FF049
:102A3000490EE66EDDEC1FF0E552030E00242A6E0F
:102A4000010114512A5C5EE2F29E939A8A9A000078
:102A50008A8C0000000000008A9C00008A8C000024
:102A6000000000008A9C00008A8C0000000000002A
:102A70008A9C00008A8C0000000000008A9C002ACA
:102A80000050EA6AA00FE96E000EEA22EFCF14F0C0
:102A9000002A0050EA6AA00FE96E000EEA22EFCF8A
:102AA00013F0002A0050EA6AA00FE96E000EEA2235
:102AB000EF500E6E180E0D6E143213320E32D8A077
:102AC0008A9AD8B08A8A00008A8C00000000000030
:102AD0008A9C0D2EF1D78A9A0D6A0D502A6E2B6AA8
:102AE000D8902B5004E68C0E2A5C000E2B5808E27E
:102AF00000008A8C0000000000008A9C0D2AEDD79F
:102B0000F28E0DD0FE0EE66EDDEC1FF0E5520028D1
:102B1000EA6AA00FE96E000EEA22040EEF6ED0EF13
:102B20001FF03F0EE66EDDEC1FF0E552002A00506C
:102B3000EA6AA00FE96E000EEA22EF500D6E3F0E1A
:102B40000D140E6E00500E240E240E242A6E010168
:102B500014512A5C01E386D0C00E0D14E76E080EF6
:102B6000E7CFDBFF080EDB50400806E11C0EF36EDA
:102B7000080EF3CFDBFF13D0080EDB50800806E110
:102B8000380EF36E080EF3CFDBFF09D0080EDB50D2
:102B9000C00805E1540EF36E080EF3CFDBFFF29E82
:102BA000939A3F0E0D14E76E070EE7CFDBFF070E7B
:102BB000DB5056E08A9A00008A8C0000000000007A
:102BC0008A9C00008A8C0000000000008A9C0000A3
:102BD0008A8C0000000000008A9C00008A8C0000A3
:102BE000000000008A9C002A0050EA6AA00FE96EEB
:102BF000000EEA22EFCF14F0002A0050EA6AA00F7C
:102C0000E96E000EEA22EFCF13F0002A0050EA6AC4
:102C1000A00FE96E000EEA22EF500E6E180E0D6E38
:102C2000143213320E32D8A08A9AD8B08A8A0000A1
:102C30008A8C0000000000008A9C0D2EF1D78A9A31
:102C4000080EDB500D6E0D5008E000008A8C00006D
:102C5000000000008A9C0D06F6D7070EDB06A7D7FA
:102C6000F28E0DD0FE0EE66EDDEC1FF0E552002870
:102C7000EA6AA00FE96E000EEA22040EEF6ED0EFB2
:102C80001FF0370EE66EDDEC1FF0E552F29E939AD0
:102C90008A8A00008A8C0000000000008A9C8A9AC0
:102CA0000D6A0B0E0D5C08E200008A8C000000002B
:102CB00000008A9C0D2AF5D7938A100E0D6E8A8C1F
:102CC000000000000000D89081BAD880143213327E
:102CD0008A9C0D2EF4D78A9AF28E14C0E6FFDDECA2
:102CE0001FF0E55213C0E6FFDDEC1FF0E552D0EF18
:102CF0001FF0380EE66EDDEC1FF0E552F29E939A5F
:102D00008A9A0D6A1C0E0D5C08E200008A8C000095
:102D1000000000008A9C0D2AF5D7F28ED0EF1FF03C
:102D2000390EE66EDDEC1FF0E552002A0050EA6A2B
:102D3000A00FE96E000EEA22EF500D6E00500D2438
:102D40000D242A6E010114512A5C48E2F29E939AE6
:102D5000090E0DC0DBFF090EDB503CE0002A0050DD
:102D6000EA6AA00FE96E000EEA22EFCF14F0002A03
:102D70000050EA6AA00FE96E000EEA22EFCF13F0CE
:102D8000100E0D6E13361436D8A08A9AD8B08A8ADF
:102D900000008A8C06C00EF00E0609E0000000005C
:102DA000000000000000000000000000F5D78A9C31
:102DB00006C00EF00E0609E0000000000000000052
:102DC0000000000000000000F5D70D2EDBD7090E33
:102DD000DB06C1D78A9A938AF28E0DD0FE0EE66E7C
:102DE000DDEC1FF0E5520028EA6AA00FE96E000E44
:102DF000EA22040EEF6ED0EF1FF03A0EE66EDDEC25
:102E00001FF0E552002A0050EA6AA00FE96E000E9A
:102E1000EA22EF500D6E01011451005C48E20150AE
:102E20000D240D242A6E400E2A5C41E20D50E66E00
:102E3000DDEC1FF0E552F29E938A0A0E0DC0DBFF17
:102E40000A0EDB5032E0100E0D6E8A8C06C00EF0BA
:102E50000E0609E000000000000000000000000075
:102E600000000000F5D7D89081BAD8801336143608
:102E70008A9C06C00EF00E0609E00000000000006B
:102E800000000000000000000000F5D70D2EDDD787
:102E900014C0E6FFDDEC1FF0E55213C0E6FFDDECE9
:102EA0001FF0E5520A0EDB06CBD7F28E0DD0FE0ED8
:102EB000E66EDDEC1FF0E5520028EA6AA00FE96E2D
:102EC000000EEA22040EEF6ED0EF1FF03B0EE66E0E
:102ED000DDEC1FF0E552C50E936E8A6A949ED0EF2A
:102EE0001FF03C0EE66EDDEC1FF0E552002A0050AC
:102EF000EA6AA00FE96E000EEA22EF500D6E0D0493
:102F00000024E8380F0B2A6E010114512A5C22E2DA
:102F1000F29E0E6A0D5000081BE20E500BE1002AD3
:102F20000050EA6AA00FE96E000EEA22EFCF13F01C
:102F3000080E0E6E1336D8A08B9ED8B08B8E8A8268
:102F400000000000000000008A920D060E06E2D785
:102F5000F28E0DD0FE0EE66EDDEC1FF0E55200287D
:102F6000EA6AA00FE96E000EEA22040EEF6ED0EFBF
:102F70001FF03D0EE66EDDEC1FF0E55200282A6ED4
:102F8000010114512A5C3AE20D040124E8380F0BC8
:102F90002B6E400E2B5C32E2002A0050EA6AA00F32
:102FA000E96E000EEA22EF500D6E0D50E66EDDEC7C
:102FB0001FF0E552F29E0001136A080E0E6E0D50CE
:102FC00000081AE28A8200000000000000008A92D5
:102FD000D89081B0D88013360E060E5002E00D0452
:102FE00009E1080E0E6E13C0E6FFDDEC1FF0E5529E
:102FF0000001136A0D06E3D7F28E0DD0FE0EE66EC9
:10300000DDEC1FF0E5520028EA6AA00FE96E000E21
:10301000EA22040EEF6ED0EF1FF0400EE66EDDECFC
:103020001FF0E552F29E8A80939000008A90FA0E7B
:10303000E66E81EC20F0E552FA0EE66E81EC20F0AF
:10304000E5528A8000009380460EE66E81EC20F007
:10305000E55281B006D0010EE66EDDEC1FF0E552C0
:1030600004D0E66ADDEC1FF0E552960EE66E81ECC8
:1030700020F0E552960EE66E81EC20F0E552F28EDD
:10308000D0EF1FF0410EE66EDDEC1FF0E552002A96
:103090000050EA6AA00FE96E000EEA22EF500D6EB2
:1030A00000500D242A6E010114512A5C3AE20D50A1
:1030B00037E0002A0050EA6AA00FE96E000EEA220B
:1030C000EF500E6EF29E080EF36E0B0EF3CFDBFF89
:1030D0000B0EDB50000821E28A9093900EA00CD0DA
:1030E000040EE66E81EC20F0E5528A80420EE66E18
:1030F00081EC20F0E5520BD03C0EE66E81EC20F026
:10310000E5528A800A0EE66E81EC20F0E5520E4010
:103110007F0B0E6E0B0EDB06DBD7F28E0D06C7D7CC
:103120000DD0FE0EE66EDDEC1FF0E5520028EA6AD7
:10313000A00FE96E000EEA22040EEF6ED0EF1FF032
:10314000420EE66EDDEC1FF0E552002A0050EA6AFE
:10315000A00FE96E000EEA22EF500D6E010114512E
:10316000005C48E201500D242A6E400E2A5C42E2C7
:103170000D50E66EDDEC1FF0E5520D503AE0F29E88
:103180000E6A080EF36E0C0EF3CFDBFF0C0EDB5055
:10319000000827E28A909390060EE66E81EC20F0FC
:1031A000E5528A8000009380080EE66E81EC20F0E4
:1031B000E5520E407F0B0E6E81A002D0800E0E26CF
:1031C000280EE66E81EC20F0E5528A809390000094
:1031D0009380100EE66E81EC20F0E5520C0EDB06BB
:1031E000D5D70E50E66EDDEC1FF0E552F28E0D06DF
:1031F000C4D70DD0FE0EE66EDDEC1FF0E5520028C0
:10320000EA6AA00FE96E000EEA22040EEF6ED0EF1C
:103210001FF0430EE66EDDEC1FF0E552F29E8A9041
:1032200093900A0EE66E81EC20F0E5528A80FA0E49
:10323000E66E81EC20F0E552FA0EE66E81EC20F0AD
:10324000E5526E0EE66E81EC20F0E5529380F28E30
:10325000D0EF1FF0440EE66EDDEC1FF0E552002AC1
:103260000050EA6AA00FE96E000EEA22EF500D6EE0
:10327000002A0050EA6AA00FE96E000EEA22EF5021
:103280000E6E00500D242A6E010114512A5C01E3D8
:10329000B5D101500E242B6E400E2B5C01E3AED154
:1032A000F29E0D5001E175D08A909390140EE66E57
:1032B00081EC20F0E5528A800A0EE66E81EC20F067
:1032C000E5528A90140EE66E81EC20F0E5528A8079
:1032D000140EE66E81EC20F0E5528A90140EE66E34
:1032E00081EC20F0E5528A80140EE66E81EC20F02D
:1032F000E5528A90140EE66E81EC20F0E5528A8049
:10330000140EE66E81EC20F0E5528A90140EE66E03
:1033100081EC20F0E5528A800A0EE66E81EC20F006
:10332000E5528A900A0EE66E81EC20F0E5528A8022
:103330000A0EE66E81EC20F0E5529380050EE66EF3
:1033400081EC20F0E5520D0EDB6A81B005D0010E54
:10335000F36E0D0EF3CFDBFF0A0EE66E81EC20F06C
:10336000E55281B005D0010EF36E0D0EF3CFDBFFF9
:10337000020EE66E81EC20F0E5520D0EDB5009E006
:10338000FD0EE66EDDEC1FF0E5520E6A0D6A0D5083
:1033900000260D5001E186D0002A0050EA6AA00FF5
:1033A000E96E000EEA220E0EEFCFDBFF8A909390BB
:1033B000080EF36E0D0EF3CFDBFF0D0EDB50000891
:1033C00020E20E0EDBAE08D08A900A0EE66E81EC8B
:1033D00020F0E5528A8007D08A800A0EE66E81ECE2
:1033E00020F0E5528A90080EE66E81EC20F0E5525E
:1033F0000E0EDB50020D0E0EF3CFDBFF0D0EDB06C3
:10340000DCD70E5003E10D50010808E28A900A0E45
:10341000E66E81EC20F0E5528A8007D08A800A0EA1
:10342000E66E81EC20F0E5528A900A0EE66E81ECA1
:1034300020F0E5529380050EE66E81EC20F0E55217
:103440000D0EDB6A81A005D0010EF36E0D0EF3CFD9
:10345000DBFF0A0EE66E81EC20F0E55281B005D06C
:10346000010EF36E0D0EF3CFDBFF0D0EDB500AE005
:10347000FD0EE66EDDEC1FF0E552010E0D6E0E6ADC
:103480000D5000260D5001080BE200000000000066
:10349000000000000000000000000000000000002C
:1034A0000D0677D70000000000000E50E66EDDEC40
:1034B0001FF0E5520E5001E19FD00E0EDB6A9380A3
:1034C000080EF36E0D0EF3CFDBFF0D0EDB50000880
:1034D0003AE2030EE66E81EC20F0E5520E0EDB5070
:1034E000020D0E0EF3CFDBFF81B00BD00A0EE66E9D
:1034F00081EC20F0E55281A003D00E0EDB2A00D033
:103500000BD00A0EE66E81EC20F0E55281A000D0CF
:1035100000000000000000000000000000000000AB
:1035200000000D0EDB50010806E2040EE66E81EC91
:1035300020F0E55205D0020EE66E81EC20F0E55257
:103540000D0EDB06C2D700000000000000000000E6
:10355000000093900E50010808E28A900A0EE66E71
:1035600081EC20F0E5528A8007D08A800A0EE66E50
:1035700081EC20F0E5528A900E0EDBCFE6FFDDEC09
:103580001FF0E552070EE66E81EC20F0E5529380C5
:10359000050EE66E81EC20F0E5520D0EDB6A81A08F
:1035A00005D0010EF36E0D0EF3CFDBFF0A0EE66EB3
:1035B00081EC20F0E55281B005D0010EF36E0D0EC6
:1035C000F3CFDBFF030EE66E81EC20F0E552000046
:1035D00000000000000000000000000000000000EB
:1035E0000D0EDB5007E0FD0EE66EDDEC1FF0E55240
:1035F000010E0E6E0E065ED7F28E0DD0FE0EE66E3A
:10360000DDEC1FF0E5520028EA6AA00FE96E000E1B
:10361000EA22040EEF6ED0EF1FF0450EE66EDDECF1
:103620001FF0E552020E00242A6E010114512A5C9B
:1036300021E2002A0050EA6AA00FE96E000EEA2299
:10364000EF50936E002A0050EA6AA00FE96E000E58
:10365000EA22EF500D6EC00E0D142A6E3F0E941428
:103660002A10946E380E0D142A6EC70E92142A106A
:10367000926E0DD0FE0EE66EDDEC1FF0E5520028D6
:10368000EA6AA00FE96E000EEA22040EEF6ED0EF98
:103690001FF0460EE66EDDEC1FF0E5528150E66E3F
:1036A000DDEC1FF0E552D0EF1FF0470EE66EDDECCB
:1036B0001FF0E552C00E82142A6E380E80142A10B4
:1036C000E66EDDEC1FF0E552D0EF1FF0480EE66E1F
:1036D000DDEC1FF0E552002A0050EA6AA00FE96E07
:1036E000000EEA22EF500D6E00500D240D242A6EBC
:1036F000010114512A5C50E2F29E8B9C8A908B9EB1
:103700009390949E949C0F0E0DC0DBFF0F0EDB5028
:103710003CE0002A0050EA6AA00FE96E000EEA229F
:10372000EFCF13F0002A0050EA6AA00FE96E000EF6
:10373000EA22EFCF14F08B8C000000008B9C080E67
:103740000D6ED89081B2D8800E361336D8A08A90EC
:10375000D8B08A801436D8A08B9ED8B08B8E00004B
:103760008B8C000000008B9C0D2EEBD78B8C000007
:1037700000008B9C000000008B8C000000008B9CE4
:103780008A908B9E0F0EDB06C1D70E50E66EDDECE5
:103790001FF0E552F28E0DD0FE0EE66EDDEC1FF04E
:1037A000E5520028EA6AA00FE96E000EEA22040E34
:1037B000EF6EF6D3530EE66EDDEC1FF0E5520028F7
:1037C0002A6E010114512A5C1AE2002A0050EA6AAA
:1037D000A00FE96E000EEA22EFCF13F0F29E13362F
:1037E00013368A9E060E0D6E1336D8A08A98D8B06E
:1037F0008A888A8C8A9C0D2EF7D7F28E0CD0FE0E0A
:10380000E66EDBDBE5520028EA6AA00FE96E000EE7
:10381000EA22040EEF6EC4D3540EE66ECEDBE55200
:1038200000282A6E010114512A5C30E2002A00505F
:10383000EA6AA00FE96E000EEA22EFCF13F0F29EC3
:103840008A9E8A888A8C8A9C8A8C8A9C8A988A8C8E
:103850008A9C8A8C8A9C040E0D6E1332D8A08A9E94
:10386000D8B08A8E8A8C8A9C0D2EF7D78A8813321C
:10387000D8A08A9ED8B08A8E8A8C8A9C8A9E8A8C8E
:103880008A9C8A988A8C8A9CF28E0CD0FE0EE66EF8
:1038900094DBE5520028EA6AA00FE96E000EEA22E6
:1038A000040EEF6E7DD3550EE66E87DBE552040EF7
:1038B00000242A6E010114512A5C65E2002A00509E
:1038C000EA6AA00FE96E000EEA22EFCF16F0002A96
:1038D0000050EA6AA00FE96E000EEA22EFCF15F061
:1038E000002A0050EA6AA00FE96E000EEA22EFCF2C
:1038F00014F0002A0050EA6AA00FE96E000EEA22D6
:10390000EFCF13F0F29E8A9E8A888A8C8A9C8A98CE
:103910008A8C8A9C8A8C8A9C1F0E0D6E16321532F8
:1039200014321332D8A08A9ED8B08A8E169E81BADD
:10393000168E8A8C8A9C0D2EF1D78A881632153203
:1039400014321332D8A08A9ED8B08A8E169E81BABD
:10395000168E8A8C8A9C8A9E8A8C8A9C8A988A8CEB
:103960008A9C16C0E6FF29DBE55215C0E6FF25DB81
:10397000E55214C0E6FF21DBE55213C0E6FF1DDB74
:10398000E552F28E0CD0FE0EE66E17DBE5520028F3
:10399000EA6AA00FE96E000EEA22040EEF6E00D371
:1039A000560EE66E0ADBE552040E00242A6E010173
:1039B00014512A5C67E2002A0050EA6AA00FE96EFF
:1039C000000EEA22EFCF16F0002A0050EA6AA00F9C
:1039D000E96E000EEA22EFCF15F0002A0050EA6AE5
:1039E000A00FE96E000EEA22EFCF14F0002A00507B
:1039F000EA6AA00FE96E000EEA22EFCF13F0F29E02
:103A00008A9E8A888A8C8A9C8A988A8C8A9C8A8CCC
:103A10008A9C8A8C8A9C1F0E0D6E163215321432C7
:103A20001332D8A08A9ED8B08A8E169E81BA168E7E
:103A30008A8C8A9C0D2EF1D78A8816321532143260
:103A40001332D8A08A9ED8B08A8E169E81BA168E5E
:103A50008A8C8A9C8A9E8A8C8A9C8A988A8C8A9C68
:103A600016C0E6FFAADAE55215C0E6FFA6DAE5526F
:103A700014C0E6FFA2DAE55213C0E6FF9EDAE55273
:103A8000F28E0CD0FE0EE66E98DAE5520028EA6A55
:103A9000A00FE96E000EEA22040EEF6E81D2570EDF
:103AA000E66E8BDAE55200282A6E010114512A5C79
:103AB00019E2002A0050EA6AA00FE96E000EEA221D
:103AC000EFCF13F0F29E939A080E0D6E13368A9A7A
:103AD000D8B08A8A8A8C00008A9C0D2EF7D78A9AE1
:103AE000F28E0CD0FE0EE66E68DAE5520028EA6A25
:103AF000A00FE96E000EEA22040EEF6E51D2580EAE
:103B0000E66E5BDAE55200282A6E010114512A5C48
:103B100043E2002A0050EA6AA00FE96E000EEA2292
:103B2000EFCF13F0F29E939A080E0D6E13368A9A19
:103B3000D8B08A8A8A8C00008A9C0D2EF7D78A9A80
:103B4000938A0D6A020E0D5C03E200000D2AFAD77B
:103B50000D6A070E0D5C06E28A8C00008A9C00004C
:103B60000D2AF7D7136A146A100E0D6E8A8CD8903E
:103B70008A9C81BAD880133614360D2EF7D78A8CDA
:103B8000939A8A9CF28E14C0E6FF17DAE55213C0AE
:103B9000E6FF13DAE5520CD0FE0EE66E0EDAE552C1
:103BA0000028EA6AA00FE96E000EEA22040EEF6E0A
:103BB000F7D1590EE66E01DAE552030E00242A6EA3
:103BC000010114512A5C46E2002A0050EA6AA00F63
:103BD000E96E000EEA22EFCF13F0F29E939A080EE0
:103BE0000D6E13368A9AD8B08A8A8A8C00008A9C15
:103BF0000D2EF7D78A9A002A0050EA6AA00FE96EC4
:103C0000000EEA22EFCF14F0002A0050EA6AA00F5B
:103C1000E96E000EEA22EFCF13F00D6A070E0D5C7D
:103C200006E28A8C00008A9C00000D2AF7D7100E4D
:103C30000D6E133614368A9AD8B08A8A8A8C0000A0
:103C40008A9C0D2EF6D78A9A8A8C00008A9C0000E6
:103C5000F28E0CD0FE0EE66EB0D9E5520028EA6A6C
:103C6000A00FE96E000EEA22040EEF6E99D1400E0D
:103C7000015C09E20150EA6A600FE96E000EEA2277
:103C8000EF6A012AF4D7016A04010CBF0BD0400E81
:103C9000E66E600EE66E000EE66E48EC21F0E55230
:103CA000E552E55200687CD1F00EE66E86D9E55209
:103CB000020E00242A6E010114512A5C25E2002A1A
:103CC0000050EA6AA00FE96E000EEA22EFCF14F06E
:103CD000002A0050EA6AA00FE96E000EEA22EFCF38
:103CE00013F014C0E6FF69D9E55213C0E6FF65D9A9
:103CF000E55214C0EAFF13C0E9FFEF500D6E0D50FE
:103D0000E66E5BD9E5520CD0FE0EE66E56D9E55252
:103D10000028EA6AA00FE96E000EEA22040EEF6E98
:103D20003FD1F10EE66E49D9E552030E00242A6E0A
:103D3000010114512A5C2EE2002A0050EA6AA00F09
:103D4000E96E000EEA22EFCF14F0002A0050EA6A72
:103D5000A00FE96E000EEA22EFCF13F0002A005008
:103D6000EA6AA00FE96E000EEA22EF500D6E14C051
:103D7000E6FF23D9E55213C0E6FF1FD9E5520D50E7
:103D8000E66E1BD9E55214C0EAFF13C0E9FF0D50DF
:103D9000EF6E0CD0FE0EE66E10D9E5520028EA6AEE
:103DA000A00FE96E000EEA22040EEF6EF9D0F30EBA
:103DB000E66E03D9E552030E00242A6E0101145168
:103DC0002A5C29E20101155126E0002A0050EA6A26
:103DD000A00FE96E000EEA22EF50F86E002A0050A4
:103DE000EA6AA00FE96E000EEA22EF50F76E002A91
:103DF0000050EA6AA00FE96E000EEA22EF50F66E5C
:103E00000900F550E66ED9D8E5520A00F550E66E85
:103E1000D4D8E5520CD0FE0EE66ECFD8E55200287D
:103E2000EA6AA00FE96E000EEA22040EEF6EB8D027
:103E3000F40EE66EC2D8E552050E00242A6E01018A
:103E400014512A5C33E20101155130E0002A005080
:103E5000EA6AA00FE96E000EEA22EF50F86E002A1F
:103E60000050EA6AA00FE96E000EEA22EF50F76EEA
:103E7000002A0050EA6AA00FE96E000EEA22EF5015
:103E8000F66E002A0050EA6AA00FE96E000EEA22E0
:103E9000EF50F56E0D00002A0050EA6AA00FE96E9F
:103EA000000EEA22EF50F56E0E000CD0FE0EE66E0C
:103EB00084D8E5520028EA6AA00FE96E000EEA22D3
:103EC000040EEF6E6DD0F50EE66E77D8E552002841
:103ED0002A6E010114512A5C14E2002A0050EA6A99
:103EE000A00FE96E000EEA22EF500101186F196B66
:103EF00018C1E6FF62D8E552002801011A6F1B6B5A
:103F00000CD0FE0EE66E59D8E5520028EA6AA00FE2
:103F1000E96E000EEA22040EEF6E42D0F60EE66E57
:103F20004CD8E55201011807000E195B18C1E6FFD5
:103F300044D8E5520101193504E218510008000E79
:103F4000195528E2400E015C09E20150EA6A600F4F
:103F5000E96E000EEA22EF6A012AF4D7016A040131
:103F60000CBF0CD0400EE66E600EE66E000EE66EE4
:103F700048EC21F0E552E552E55203D00001010E74
:103F8000EA6F1AC12AF01BC12BF02A06000E2B5A29
:103F90002A50006E05D0FE0EE66E0FD8E55200D016
:103FA000002A01D08992100EE15C02E2E16AE5523A
:103FB000E16EE552E7CFD9FF1200D9CFE6FFE1CF9E
:103FC000D9FF0001EA510AE00A0E025C11E2025038
:103FD000022AEA6AE00FE96E000E06D00150012ABB
:103FE000EA6A600FE96E000EEA22FE0EDBCFEFFFF9
:103FF000400E015C13E1016A04010CBF0CD0400EBD
:10400000E66E600EE66E000EE66E48EC21F0E552BC
:10401000E552E55203D00001010EEA6FE552E7CF09
:10402000D9FF1200D8CFE4FFE0CFE4FFE46EDACF8F
:10403000E4FFE2CFDAFFF3CFE4FFF4CFE4FFE65290
:10404000C2B2FED79E9C07C009F008C00AF0C4CFD8
:1040500008F0C3CF07F00B50075E0C50085AE10E72
:104060000902F4CF10F0F3CF0FF0E10E0A02F35083
:1040700010260F50032610500422E40E0702F4CF3E
:1040800010F0F3CF0FF0E40E0802F35010260F509B
:10409000035E1050045A043404E303500008FE0E7B
:1040A000045403E3036AFE0E046E043404E2035076
:1040B0000008640E045403E2036A640E046E0001F7
:1040C000043405E3BE6ACF0EBD14BD6E0DD004C02E
:1040D000BEFF00010350E840E8403F0B300B2E6E5E
:1040E000CF0EBD142E10BD6EE552E5CFF4FFE5CF27
:1040F000F3FFE5CFDAFFE550E5CFE0FFE5CFD8FFEE
:104100001000D9CFE6FFE1CFD9FFE652FE0EDB501B
:10411000FE0FDF6EDF5009E000000000000000002D
:10412000000000000000DF06F5D700D0E552E552A0
:10413000E7CFD9FF12008A90939001EF21F08A9285
:10414000939293805ED893825CD881B0FF0C000C70
:10415000080E186E8A929392938053D8938251D806
:10416000179E1746179081B017801806F4E12B6A46
:1041700017C0F3FF2BC0F4FF1200D9CFE6FFE1CF49
:10418000D9FF080E186EFE0EDB50176E8A92173696
:10419000D8A006D09392938034D8938232D806D098
:1041A00093928A9093902DD893822BD8180618500A
:1041B000EEE1000E00D0E552E7CFD9FF12008A925F
:1041C000939293801ED893821CD88A90939001EF8B
:1041D00021F08A9293928A90939013D8938211D867
:1041E00093800FD801EF21F0939293800AD89382A5
:1041F00001EF21F093928A90939003D8938201EF7C
:1042000021F0ECC019F0195009E000000000000096
:1042100000000000000000001906F5D700D01200D1
:10422000D9CFE6FFE1CFD9FFF29EFE0EDB50176E2D
:10423000ECC00FF0080E0E6E0FB404D017AE8B9EBC
:1042400017BE8B8E0650196E192EFED70FA68A82C6
:104250000FB68A920FA405D017AE8B9E17BE8B8E19
:1042600002D0813017360650196E192EFED70FA6D0
:104270008A920FB68A820FA402D0813017360E2E92
:10428000DBD7F28E175000D0E552E7CFD9FF1200EE
:10429000D9CFE6FFE1CFD9FFE65204010CAF02D03F
:1042A000000E33D0FC0EDB50400805E2400EF36EEA
:1042B000FC0EF3CFDBFFDF6AFC0EDB50DF5C19E2A4
:1042C000DF50E76EFD0EDBCFE9FFFE0EDBCFEAFF2E
:1042D000E750E926000EEA22EF50E66EDF50EA6A68
:1042E000580FE96E050EEA22E552E750EF6EDF2A1D
:1042F000E3D7FC0EDBCF0DF404010CAD02D0880E29
:1043000001D0C80E0C6FFC0EDB50E552E552E7CF32
:10431000D9FF1200D9CFE6FFE1CFD9FF0101136B1E
:10432000040108BF32D0FC0EDBCF2AF00951D8803F
:104330002A5403E2FC0E09C4DBFF0101136BFC0EDF
:10434000DB50135D19E21351EA6A180FE96E050E8E
:10435000EA22EF50E66E1351E76EFD0EDBCFE9FF68
:10436000FE0EDBCFEAFFE750E926000EEA22E55217
:10437000E750EF6E132BE3D70401400E096F08AD31
:1043800002D0880E01D0C80E086F01011351E5520A
:10439000E7CFD9FF12000101136B1E0E716E0401ED
:1043A000400E096F180E2A6E050E2AC00AF40B6F14
:1043B000880E086F580E2A6E050E2AC00EF40F6F75
:1043C000400E0C6F1200D9CFE6FFE1CFD9FFE652C5
:1043D00002C5DFFF0101010E076FE552E552E7CF8D
:1043E000D9FF1200D9CFE6FFE1CFD9FFE65202C5CF
:1043F000DFFF0101010E076FE552E552E7CFD9FF5C
:104400001200D9CFE6FFE1CFD9FF020EE1261F0E41
:1044100005010015010865E1045163E101C5DFFFF5
:10442000060EDF5C23E1010E03C5DBFFDB50210834
:1044300009E10101010E076F5D0E0A6F4C0E0B6F53
:10444000090E0CD0010EDB5022080DE10101010E16
:10445000076F7D0E0A6F4C0E0B6F220E0E6F0F6BE7
:10446000010E106F03D0010EDB502308600E050112
:104470000015200836E1DF0402E1A5DF32D0090E85
:10448000DF5C05E10101010E066FACDF2AD0020EF0
:10449000DF5C07E10101010E076F110E086F010ECD
:1044A00012D00A0EDF5C06E10101010E076F03C5A1
:1044B00011F117D0030EDF5C0CE10101010E076F53
:1044C000120E086F010E096F010E0E6F0F6B106B4D
:1044D00008D00B0EDF5C05E10101010E076F02C57C
:1044E00012F1020EE15C02E2E16AE552E16EE55290
:1044F000E7CFD9FF1200D9CFE6FFE1CFD9FF020EF7
:10450000E126800E0501005D3CE103C5DFFF010EE1
:1045100002C5DBFFDF0409E10101010E076F420E56
:104520000A6F4C0E0B6F120E28D0020EDF5C09E1F1
:104530000101010E076F540E0A6F4C0E0B6F290E0E
:104540001CD0030EDF5C1DE10101010E076FDB5083
:1045500004E19F0E0A6F4C0E0AD0010EDB0404E149
:10456000A30E0A6F4C0E03D0C30E0A6F4C0E0B6FD6
:104570000AC1F6FFF76E0800F5500E6F0F6B010EC3
:10458000106F020EE15C02E2E16AE552E16EE55273
:10459000E7CFD9FF1200D9CFE6FFE1CFD9FF030E55
:1045A000E1261F0E05010015DF6E106B116BDF5049
:1045B0000DE10101010E076F035102E005011081B9
:1045C0000101015135E00501108332D0DF0404E11F
:1045D0000101010E076F2CD0020EDF5C29E10F0EE6
:1045E0000415E76E010EE7CFDBFF800E0415E76EC2
:1045F000020EE7CFDBFF0101010E076FDB50080D54
:10460000F3500C6F0D6B000E0C27040E0D23020EE1
:10461000DB5004E0040E0C27000E0D230CC1E9FF53
:104620000DC1EAFFEF50040B03E00501010E106F0E
:104630000101075108E0100E086F050E096F020E08
:104640000E6F0F6B106B030EE15C02E2E16AE55244
:10465000E16EE552E7CFD9FF1200D9CFE6FFE1CFF7
:10466000D9FF040EE1261F0E05010015DF6E010EB5
:1046700002C5DBFFDF5011E1010EDB044CE101015B
:10468000010E076F030E0501015D04E10101010E3A
:10469000016F41D00101016B3ED0020EDF5C3BE1B6
:1046A0000F0E0415E76E020EE7CFDBFF800E041538
:1046B000E76E030EE7CFDBFF010EDB502CE1020EAD
:1046C000DB5029E00101010E076F020EDB50080DDF
:1046D000F3500C6F0D6B000E0C27040E0D23030E10
:1046E000DB5004E0040E0C27000E0D23030E050121
:1046F000015D02E1840E0AD0030EDB0406E10CC169
:10470000E9FF0DC1EAFFEF6A06D0880E0CC1E9FF90
:104710000DC1EAFFEF6E040EE15C02E2E16AE552D0
:10472000E16EE552E7CFD9FF1200D9CFE6FFE1CF26
:10473000D9FFE65201C5DFFF600E0501001554E107
:10474000050EDF5C08E10101010E076F040E006F2A
:1047500002C502F149D0060EDF5C02E1CCDE44D096
:10476000090EDF5C0EE10101010E076F02C504F1C5
:10477000045103E1040E006F37D0050E006F0BDE0D
:1047800033D0080EDF5C07E10101010E076F040E54
:10479000086F010E17D0DF5002E1FDDE25D0DF04E7
:1047A00003E0030EDF5C02E158DF1ED00A0EDF5C7F
:1047B0000FE10101010E076F0501106B0101100EE1
:1047C000086F050E096F010E0E6F0F6B106B0CD08A
:1047D0000B0EDF5C04E10101010E076F05D0070E2F
:1047E000DF5C02E00C0EDF5CE552E552E7CFD9FF5B
:1047F0001200D9CFE6FFE1CFD9FF030EE126010178
:10480000080E0E5D000E0F5907E2010E0EC1DBFF10
:10481000020E0FC1DBFF07D0080EF36E010EF3CFBF
:10482000DBFF020EDB6AFC0E04010417010E020E10
:10483000DBCF2BF0000E030E2B162BC02AF02B50D3
:104840000413FF0EE76E010EDBCF2AF0020EE750D5
:104850002A162AC005F4100E2A6E050E2D6A2AC0EB
:1048600006F4076F010EDB5001010E5F020EDB50F4
:104870000F5B100E0C6F050E0D6F100524E1DF6A43
:10488000DFCF2AF0010EDBCF2BF0020EDBCF2CF0B6
:104890002B502A5C000E2C5439E20AC1F6FF0BC1E2
:1048A000F7FF0A2B000E0B230800F550E66E0CC133
:1048B000E9FF0DC1EAFF0C2B000E0D23E552E75076
:1048C000EF6EDF2ADDD7DF6ADFCF2AF0010EDBCF04
:1048D0002BF0020EDBCF2CF02B502A5C000E2C5458
:1048E00015E208C1E9FF09C1EAFF082B000E092300
:1048F000EF50E66E0CC1E9FF0DC1EAFF0C2B000E74
:104900000D23E552E750EF6EDF2ADED7030EE15CA0
:1049100002E2E16AE552E16EE552E7CFD9FF12000B
:10492000D9CFE6FFE1CFD9FF040EE126030E040143
:104930000015F3500111E66ED950020FE96EDACF7F
:10494000EAFFE552E750EE6EED6A020EDB50010120
:104950000E27030EDB500F23100E086F050E096F94
:10496000DE6ADD6ADECF2AF0DDCF2BF0020EDBCF70
:104970002CF0030EDBCF2DF02C502A5C2D502B5841
:1049800018E208C1E9FF09C1EAFF082B000E09235C
:10499000EF50E66E0CC1E9FF0DC1EAFF0C2B000ED3
:1049A0000D23E552E750EF6EDF2A010EDBE3DB2A31
:1049B000D9D7040EE15C02E2E16AE552E16EE5520C
:1049C000E7CFD9FF12000401049F009F0101056B8E
:1049D000076B066B0E6B0F6BA8DE13DD0101075131
:1049E0000EE10401080E016F000E2A6E050E2C6AFE
:1049F0002D6A2AC002F4036F840E006F30D00501C7
:104A000000AF2FD001010E510501065D01010F51CC
:104A10000501075904E206C50EF107C50FF1E9DEED
:104A20000101020E056F0401080E016F000E2A6ECF
:104A3000050E2B6E2C6A2D6A2C6A2D6A2AC002F490
:104A4000036F800E006F100E2A6E050E2B6E2C6AFF
:104A50002D6A2C6A2D6A2AC006F4076FC80E046FEF
:104A600016D00101010E056F0401056BC80E046F1D
:104A7000080E016F100E2A6E050E2B6E2C6A2D6A21
:104A80002C6A2D6A2AC002F4036FC80E006F6D985D
:104A900012000101056B0401080E016F000E2A6E61
:104AA000050E2AC002F4036F880E006F046B12001B
:104AB000D9CFE6FFE1CFD9FF020EE1266C5024E109
:104AC0003C0E04010015E840E8403F0BDF6E0D0E80
:104AD000DF5C02E178DF35D00101050531E120DF3F
:104AE0000101065109E0010E02C5DBFF020E0501BE
:104AF000035D02E0030E035D040100AD02D0880EE9
:104B000001D0C80E006F1DD0040E6C5C1AE16E500F
:104B10000AE1040E0101005D06E102C56EFF6E5060
:104B200002E1030E006F020E0101055D09E161DE85
:104B3000040104AD02D0880E01D0C80E046F01D06C
:104B4000A8DF020EE15C02E2E16AE552E16EE552A5
:104B5000E7CFD9FF12006DB606D06D6A696A6D861F
:104B60000101010E006F0101000509E16D50200BEC
:104B700006E1686A696A69806988020E006F12003E
:104B80006D92699468941200689C120070A002D023
:104B900080DF7090689A120012006A6A686A9F0E3D
:104BA0006B6E7B0E696E6E6A160E706E68A602D012
:104BB0006896FCD76D986DDF0101016B036B046B88
:104BC000030E006F12000101005101E11200685054
:104BD000040B04E06950040B01E0D2DF6DB2120057
:104BE0006850010B04E06950010B01E0D6DF68500A
:104BF000100B04E06950100B01E0CEDF6850400B51
:104C000004E06950400B01E0BFDF6850200B04E076
:104C10006950200B01E0BADF6850020B04E06950D4
:104C2000020B01E06892030E0101005D01E2120037
:104C30006850080B05E06950080B02E039DF689600
:024C4000120060
:0E4C42001201000200000008091232540100A5
:104C50000102000109022900010100A0320904003B
:104C600000020300000009210101000122220007C7
:104C70000581034000010705010340000106A0FF74
:104C80000901A1010903150026FF0075089540815F
:104C9000020904150026FF00750895409102C00422
:104CA00003090420034F00700065006E00200050CF
:104CB0000072006F006700720061006D006D00659A
:104CC0000072003E034F00700065006E002000502F
:104CD0000072006F006700720061006D006D00657A
:104CE00000720020002000550053004200200048C0
:104CF0000049004400200063006C006100730073F1
:014D000000B2
:0E4D02002A0EF66E000EF76E000EF86E00011F
:104D10000900F550F86F0900F550F96F03E1F867E5
:104D200001D03DD00900F550F36F0900F550F46F44
:104D30000900F550F56F09000900F550E96E09000A
:104D4000F550EA6E090009000900F550F66F0900F8
:104D5000F550F76F09000900F6CFFAF0F7CFFBF036
:104D6000F8CFFCF0F3C0F6FFF4C0F7FFF5C0F8FF92
:104D70000001F65302E1F75307E00900F550EE6E2B
:104D8000F607F8E2F707F9D7FAC0F6FFFBC0F7FF1E
:104D9000FCC0F8FF0001F807000EF95BBFD7120056
:104DA0001A6A28AED9EF26F0276C281EE86A282256
:104DB0001A1E23AEE1EF26F0226C231EE86A23229E
:104DC0001A1EF6EC26F023BEF1EF26F01AAE000C08
:104DD000226C231EE86A23221E6C1F1EE86A1F2213
:0C4DE000000C1ABEE8EF26F01B88FF0C48
:044DEC001F6A1E6AB2
:104DF000100EE76ED890223623361E361F36275007
:104E00001E5C28501F5805E327501E5E28501F5A6D
:084E1000222AE72EF0D7120060
:084E180022EC00F0140E6F6E95
:104E20000101006B0101016B0101046BABEC25F08A
:0E4E30006FBE02D0E3EC25F067EC00F0F7D780
:024E3E00000E64
:104E4000F36E00EE00F0080E01D81200EA6002D006
:0E4E5000EE6AFCD7F350E9601200EE6AFCD760
:024E5E0013EE51
:104E600000F023EE00F0F86A1B9C81EC26F03DEC8C
:0A4E700027F00CEC27F0FBD712002E
:024E7A00120024
:044E7C000000000032
:104E800000640100000000AB03000000000000000F
:064E90000000000000001C
:084E9600000000000000000014
:020000040030CA
:0100000022DD
:010001000EF0
:010002003DC0
:010003001EDE
:0100050000FA
:010006008178
:010008000FE8
:01000900C036
:01000A000FE6
:01000B00E014
:01000C000FE4
:01000D0040B2
:0200000400F00A
:100000004F70656E2050726F6772616D6D65722002
:10001000762E2000302E31322E3000202D20436FDE
:10002000707972696768742028432920323030392A
:100030002D3230323220416C626572746F204D6116
:100040006363696F6E69202D20546869732069733A
:0F005000206672656520736F6674776172650054
:00000001FF
